:03000000020055A6
:0300030002103DAB
:03000B00020EE7FB
:03001300020EE7F3
:03001B0002002BB5
:03002300020FA326
:10002B0032416C636F726E204D634272696465205E
:10003B00496E632E20444D58202D205665727369EE
:0A004B006F6E20352E33392020207F
:10005500C2AF75D00075812F75B81075A813787F5C
:10006500E4F6D8FD758DFD758BFD758C88758A0850
:10007500758921758804756A887569087598C0122F
:1000850008697E007F789000007400F0A3DEFCDF35
:10009500FA900000120EC9FAA3120EC9FBA3120EA4
:1000A500C9FCA3120EC9FD4C601AA3120EC9F56E48
:1000B500A3120EC9F56DA3120EC9F57E90000212AA
:1000C5000841600E7455F599780000D8FDD20302F9
:1000D500015774AAF599780000D8FDC20390000F66
:1000E500120EC9757520757400757B00757A0A85C1
:1000F5007E7FE57E605C900020A3A3D57FFB858293
:100105007385837275A0087800857E7F120EC9F20B
:10011500A308120EC9F2A308B8000205A0D57FEC0A
:10012500857E7F85758285748312059EA3A3120E35
:10013500C9540F857B82857A83F0A385827B85836D
:100145007A857582857483A3A3858275858374D525
:100155007FD1D28CD28E120DCCD29CD2AF75D00865
:100165009014007F11A3E0F8A3E0F9686003120181
:100175008D75D00010010280E4200309300A0312B6
:1001850003EC120329020162AC83AD828F8389825D
:1001950075D00075A0137800E0FB75F000E425F03C
:1001A500F5F00582E58265086024E0F208DBEF05DD
:1001B50082C5F003547FB5F015858209901300E0E0
:1001C500FBA3D2091205C075D008898280050000FD
:1001D50075D008E5828C838D82F022C082C083C0F1
:1001E500F0E5822407F582E5833400F583120EC914
:1001F500F8A3120EC9541F2410F975A014E3F9EEE3
:1002050030E708E8541F2410F8E2F8EE540F2323D2
:10021500900219730202590002025D0002026B008E
:10022500020279000202890002029B000202AB0071
:1002350002025D0002026B000202790002028900DF
:1002450002029B000202AB000202590002025900A1
:1002550002025900C30202BDE988F0B5F004D302D9
:1002650002BDC30202BDE988F0B5F004C30202BDB8
:10027500D30202BDE988F0B5F0004004C30202BD17
:10028500D30202BDE988F0B5F00280064004C3023E
:1002950002BDD30202BDE889F0B5F00040E2C30219
:1002A50002BDD30202BDE889F0B5F0028006400424
:1002B500C30202BDD30202BDD0F0D083D08222C0DA
:1002C50082C083C0F0E5822407F582E5833400F51A
:1002D50083120EC9F8A3120EC9541FF990143025C4
:1002E50082F582E0C2046002D204EE30E719E854D8
:1002F5001FF89014302582F582E06002D20475A0C3
:1003050014741028F8E2F830041275A0147410293A
:10031500F9E3F9EE540F232390021973C3D0F0D0FB
:1003250083D08222857E7FE57E70030203EB757B99
:1003350000757A0A757D00757C08857377857276F8
:1003450075710075700B857B82857A83E030E25785
:100355008571828570831205B1A38570A0A871E5AA
:1003650082F208E583F2857D82857C831205B1855D
:10037500827985837812059EE58245836019120589
:10038500766017A3A3C2091205C020060D857982E0
:10039500857883A3A380D8120548857D82857C83D3
:1003A500E579F0A3E578F0D57F02803A857B8285F3
:1003B5007A83A385827B85837A857D82857C83A3E9
:1003C500A385827D85837C857782857683A3A385B6
:1003D5008277858376857182857083A3A3858271F3
:1003E50085837002034B22901450E070030205458B
:1003F500F57F757D00757C0D857D82857C83E0F9B3
:10040500A3E0FAA3E0A3A385827D85837C89828A04
:1004150083F575C0F075F002A4F57B85F07AD0F010
:10042500A3A3120EC9FBA3120EC9FCA3120EC9FD8C
:10043500A3120EC9FEA3120EC9FFEE541FB4070086
:10044500405E1202C440028057900A00E57525827D
:10045500F582E030E24430E043E57B2400F582E5B7
:100465007A340BF5831205B1E582C39CE5839D5073
:1004750003020531120548900A00E5752582F582CB
:10048500EBD2E2F0E57B2400F582E57A3408F583CA
:10049500E579F0A3E578F0020531D2E2F002053105
:1004A500A3120EC9FEA3120EC9FFEE541FB4070016
:1004B50040171202C440028010900A00E57525829B
:1004C500F582E0C2E2F0020531A3120EC9FEA312C5
:1004D5000EC9FFEE541FB4070040171202C44002B4
:1004E5008010900A00E5752582F582E0D2E3F002DE
:1004F5000531A3120EC9FEA3120EC9FFEE541FB497
:10050500070040281202C440028021120548900AC3
:1005150000E5752582F582EBF0E57B2400F582E5A3
:100525007A3408F583E579F0A3E578F0D57F030201
:10053500053A0203FD7E209014307400F0A3DEFC22
:10054500C20A2285778285768312059E8582798502
:1005550083788570A0A8717400F208F2857B828586
:100565007A83E030E10510E3028002C2E2C2E4F0E2
:1005750022AD82AE8312059EAB82AC8385718285E6
:1005850070831205B1E582C39BE5839C400474FF2B
:10059500800274008D828E8322C0F0120EC9F5F0A0
:1005A500A3120EC9F58385F082D0F022C0F0E0F5E4
:1005B500F0A3E0F58385F082D0F022C206AD82AECD
:1005C500837A00120ED5FFA3120ED590103E75F05A
:1005D50002A42582F582E5F03583F583E493F5F0F1
:1005E500A3E49385F083F582E4730206C10206C194
:1005F5000206C10206C10206C10206C11206C602F2
:1006050006C11206F70206C10206C112070F02064D
:10061500C10206C10206C11207240206C112073D26
:100625000206C11207560206C112076F0206C11261
:1006350007CE0206C10206C1120C9C0206C10206C3
:10064500C10206C112089C0206C11208C00206C1F9
:100655001208EC0206C11209190206C112094A0262
:1006650006C11209790206C11209AC0206C11209B6
:10067500DD0206C1120A040206C1120A2D0206C1D4
:10068500120A590206C1120A8A0206C1120ABD02DD
:1006950006C1120AF40206C1120B290206C1120B89
:1006A500620206C1120B990206C1120BC80206C1ED
:1006B5000206C10206C1120C610206C18D828E833B
:1006C50022901408E0F8A3E0F5F075A0129010DE72
:1006D5007900E993600BF20908E8B5F0F5D20680D8
:1006E50010901408E8C2ACF0200804D208D299D2C0
:1006F500AC228D828E83A3A3120ED5FAA3120ED53A
:10070500FBA3120D636002D206228D828E83A3A302
:10071500120ED5547F232579F57950020578228D5F
:10072500828E83A3A3120ED5F8C3957E50097583D7
:100735000A8882E0D2E2F0228D828E83A3A3120E74
:10074500D5F8C3957E500975830A8882E0C2E2F028
:10075500228D828E83A3A3120ED5F8C3957E5009F0
:1007650075830A8882E0D2E3F0228D828E83A3A36B
:10077500120ED5F8C3957E504F857283E875F00249
:10078500A42573F582E5F03583F58312059EAB82CA
:10079500AC83758308E875F002A4F582E5F035832E
:1007A500F583EBF0A3ECF075830BE875F002A4F587
:1007B50082E5F03583F583E4F0A3F075830A88823A
:1007C500E0C2E2C2E4F0C2E322C2AF8D828E83A30F
:1007D500A3120ED5FAA3120ED5FBE599C29874AAF9
:1007E500D29BC299F599900000787079103098FDE8
:1007F500A699C298DA04EB60121B08D9F0787079D3
:1008050010E6120EB9A308D9F880DE7A007B20DA4B
:10081500FEDBFC78707910E6120EB9A308D9F80250
:100825000055F95407C90303035403C0E07401B923
:100835000002800323D9FDF9D0E0C92278007900B0
:10084500120EC928500109F8A3DC05BD00F2800687
:10085500BCFFED1D80EAE86A7007E96B7003E48070
:100865000274FF227480907803F07402907800F08F
:100875007400907801F07407907803F074C1907853
:1008850002F07400907801F07400907804F090788C
:1008950005E0907806E0228D828E83A3A3120ED503
:1008A500541FF92410F8A3120ED575A014F275A0E3
:1008B50014743029F874FFF2D20A228D828E83A334
:1008C500A3120ED5541FF92410F875A014E2F5F003
:1008D500A3120ED5B5F00FA3120ED5547F2325799B
:1008E500F57950020578228D828E83A3A3120ED549
:1008F500541F2410F875A014E2F5F0A3120ED5B517
:10090500F002800FA3120ED5547F232579F5795077
:10091500020578228D828E83A3A3120ED5541F243F
:1009250010F875A014E2F5F0A3120ED5C5F0B5F0D8
:10093500004002800FA3120ED5547F232579F57947
:1009450050020578228D828E83A3A3120ED5541FE3
:100955002410F875A014E2F5F0A3120ED5B5F00039
:100965004002800FA3120ED5547F232579F57950C7
:10097500020578228D828E83A3A3120ED5541F24DF
:1009850010F875A014E2F5F0A3120ED5C5F0B5F078
:100995000280044002800FA3120ED5547F232579CF
:1009A500F57950020578228D828E83A3A3120ED588
:1009B500541F2410F875A014E2F5F0A3120ED5B556
:1009C500F00280044002800FA3120ED5547F232528
:1009D50079F57950020578228D828E83A3A3120EB4
:1009E500D5541FF92410F875A014E2FAA3120ED5F8
:1009F5002AF275A014743029F974FFF3D20A228DF6
:100A0500828E83A3A3120ED5541FF92410F875A066
:100A150014E2FAA3120ED5CAC39AF275A014743063
:100A250029F974FFF3D20A228D828E83A3A3120EB5
:100A3500D5541FF5F02410F8A3120ED5541F241019
:100A4500F975A014E3F275A014743025F0F874FF5D
:100A5500F2D20A228D828E83A3A3120ED5541F24AF
:100A650010F875A014E2F5F0A3120ED5541F24104A
:100A7500F9E3B5F00FA3120ED5547F232579F57947
:100A850050020578228D828E83A3A3120ED5541FA2
:100A95002410F875A014E2F5F0A3120ED5541F2406
:100AA50010F9E3B5F00280DCA3120ED5547F23259F
:100AB50079F57950020578228D828E83A3A3120ED3
:100AC500D5541F2410F875A014E2F5F0A3120ED525
:100AD500541F2410F9E3C5F0B5F0004002800FA3C0
:100AE500120ED5547F232579F57950020578228D8C
:100AF500828E83A3A3120ED5541F2410F875A0145B
:100B0500E2F5F0A3120ED5541F2410F9E3B5F00059
:100B15004002800FA3120ED5547F232579F5795015
:100B2500020578228D828E83A3A3120ED5541F242D
:100B350010F875A014E2F5F0A3120ED5541F241079
:100B4500F9E3C5F0B5F00280044002800FA3120E50
:100B5500D5547F232579F57950020578228D828E2B
:100B650083A3A3120ED5541F2410F875A014E2F523
:100B7500F0A3120ED5541F2410F9E3B5F00280043A
:100B85004002800FA3120ED5547F232579F57950A5
:100B9500020578228D828E83A3A3120ED5541FF5EC
:100BA500F02410F875A014E2FAA3120ED5541F24F0
:100BB50010F9E32AF275A014743025F0F874FFF2E9
:100BC500D20A228D828E83A3A3120ED5541FF5F06F
:100BD5002410F875A014E2FAA3120ED5541F2410A0
:100BE500F9E3CAC39AF275A014743025F0F874FFBE
:100BF500F2D20A227A007B007C00601675F00A8426
:100C0500AAF0600E75F00A84ABF0600675F00A84F0
:100C1500ACF0EA2430FAEB2430FBEC2430FC2290D3
:100C25000000120EC9FB902000120EC9FDEBF41254
:100C35000EB9120C91120EC9F4B5030E90000012F4
:100C45000EC9B503057A20020C517A08902000EDF3
:100C5500120EB9120C91901451EAF022120C249044
:100C65001451E0FA901408E0F8A3E0F5F075A0122D
:100C7500EAF208E8B5F004D2068010901408E8C23C
:100C8500ACF0200804D208D299D2AC227C0075F0D1
:100C950019DCFED5F0FB22EFB56E028003020D2DA7
:100CA5008D828E83A3120ED5FFA3120ED5FAA31241
:100CB5000ED5FBBF0907A3120ED5F9800279009066
:100CC5000000EA75F008A42582F582E5F03583F584
:100CD50083A3A3A3E0F88BF0B90008E5F0F0A3F037
:100CE500020D2DA3E5F0F0E8B5F003020D2D400649
:100CF500E8C395F08004E5F0C39889F0B5F000509D
:100D050015C5F084F8E58254F8F582E8F0A3E8F01B
:100D1500A37401F0801284F8E58254F8F582740119
:100D2500F0A37401F0A3E8F022E0F8A3E0FDA3E04E
:100D3500CDB51503020D624003020D4B284012B5D7
:100D45001500500D8009C3984007B5150040028075
:100D550001EDFDE58254F84403F582EDF022AE8203
:100D6500AF83901408EA2323232582F58274003586
:100D750083F583E0F8A3E0F9EA2412F5A089F08E63
:100D8500828F83120ED5F2A308E8B5F003020DC5D4
:100D9500DBF1AE82AF83901408EA2323232582F585
:100DA5008274003583F583E8BA000FC2ACF02008E1
:100DB50004D208D299D2AC020DBFE48E828F832271
:100DC50074FF8E828F832290000A20033B120EC986
:100DD500600DC2A9D2AAF568856867D2078039C2B5
:100DE50007900009120EC9B40008756A6A7569088A
:100DF500801CB40108756A877569E98011B4030818
:100E0500756A707569088006756A88756908856AE6
:100E15008C85698AC2AAD2A9D20222E57E70030214
:100E25000EB8857E7F7A007B007800790D75752078
:100E350075740085758285748312059EAE82AF83B5
:100E450074052582F58274003583F5837C04C2041C
:100E5500C205120EC9A36002D204120EC9A3B4FFC3
:100E6500028002D205DCEB30041788828983EEF01C
:100E7500A3EFF0A3E57EC3957FF0A3A3A882A98382
:100E85000B3005198D8285F083EEF0A3EFF0A3E515
:100E95007EC3957FF0A3A3AD828583F00A85758215
:100EA500857483A3A3858275858374D57F85901406
:100EB50050EBF022C0E0AE83E5832480F583D0E0DB
:100EC500F08E8322C083E5832480F583E0D08322DE
:100ED500300903E0800BAE83E5832480F583E08E43
:100EE5008322D290C290C0D0C0E0C083C08275D0AA
:100EF500107447907803C2AFF07F26DFFE74079029
:100F05007803F0D2AF756600C0A075A07878007937
:100F150005E4F2900003E330E5FCE0F2E582240805
:100F2500F582E5833400F5830566E56670E8D0A0B3
:100F350075660090FFFCE5822407F582E5833400A1
:100F4500F583E0F8A3E0B51009E56604F56670E6FB
:100F5500801EC082C083E58254F8F582E0F8A3E0E4
:100F650014F07006E8F0A3120D2ED083D08280D93C
:100F750030020FD201856B83856C82A385836B85D7
:100F8500826C200710C28CE58A2569F58AE58C35C7
:100F95006AF58CD28CD082D083D0E0D0D032C0D04C
:100FA500C0E0C083C08275D01820980F3099030225
:100FB5001019D082D083D0E0D0D032C298901401DD
:100FC500E0F8A3E0F9A3E0FAA3E0FBE599FF309A86
:100FD5001030E70DC29A7B01E8FA0AEA6970027BD4
:100FE50000EB60217583118A82EFF00582E5826945
:100FF50070047B00800FAA820B309A098882EB145B
:10100500F0EAF87B00901401E8F0A3A3EAF0A3EB63
:10101500F0020FAEC299901408E0F8A3E0B51805E8
:10102500C208020FAE758312F582E0F5990582E5D7
:1010350082901409F0020FAE3206C106C105EF0514
:10104500F205F505F805FB063D06C1063D06C10698
:10105500C105FE060706100616061906C1060D0689
:10106500C106C106C106C106C1061C062206280620
:101075002E063A06C106C106C106B506C1064306D7
:101085004606C106C106C106C10649064F065506F4
:101095005B06610667066D06730679067F0685069B
:1010A5008B06910697069D06A306A906AF06B80608
:1010B500C106BB06C106C106C1063406C106010646
:1010C500C106C106C106C106C106C106C106C106E3
:1010D500C106C106C106C106C1444D582056352E6C
:0410E50033390D008E
:00000001FF
